:10000000789D001001010000090100005F0A000056
:10001000291B000051020000293100007C07FFEF7E
:1000200000000000000000000000000013010000BC
:100030001501000000000000170100002926000043
:100040001B0100001B010000AD2600001B01000089
:100050001B0100001B0100001B0100001B01000030
:100060001B0100001B0100001B0100001B01000020
:100070001B010000000000001B0100001B0100002C
:100080001B0100001B0100001B0100001B01000000
:100090001B0100001B0100001B0100001B010000F0
:1000A000992A00001B0100001B0100001B01000039
:1000B0001B0100001B0100001B0100001B010000D0
:1000C0001B0100001B0100001B0100001B010000C0
:1000D0001B0100001B0100001B0100001B010000B0
:1000E0001B010000DFF80CD000F062F80048004768
:1000F0008D380000789D0010D0F800D0D0F804F0C2
:100100000648804706480047FEE7FEE7FEE7FEE7B1
:10011000FEE7FEE7FEE7FEE7FEE7FEE74526000016
:10012000E500000010B50B4604461146184600F0E5
:100130002BF8C4E9000110BD40EA01039B0703D07E
:1001400009E008C9121F08C0042AFAD203E011F816
:10015000013B00F8013B521EF9D2704730B50B4607
:10016000014600202022012409E021FA02F59D42E7
:1001700005D303FA02F5491B04FA02F52844151EBB
:10018000A2F10102F1DC30BD70B500242546002843
:1001900001DA01244042002901DA01254942FFF732
:1001A000DDFFAC4200D04042002C00D0494270BD7F
:1001B000064C074D06E0E06840F0010394E80700B4
:1001C00098471034AC42F6D3FFF790FF9C420000F2
:1001D000BC42000070B58C1810F8015B15F00703E5
:1001E00001D110F8013B2A1106D110F8012B03E0D0
:1001F00010F8016B01F8016B5B1EF9D12B0705D4D8
:100200000023521E0DD401F8013BFAE710F8013B20
:10021000CB1A921C03E013F8015B01F8015B521E3C
:10022000F9D5A142D8D3002070BD10B50C460022EC
:1002300000F026FC4FF0402188680A3404EB4402A9
:10024000C2EBC4128B681B1AB3EBC20FFAD310BDFA
:10025000032000F0E9FB000070B50023084D0AE020
:10026000CE5C04885B1C86EA14269BB235F81660C7
:1002700086EA04240480521E92B2F1D270BD0000BE
:10028000843D00002DE9FC410746002090460E46C3
:10029000ADF8000004460EE0351B402D00D9402586
:1002A00039192A460D4800F067FFAAB20B49684683
:1002B000FFF7D2FF2C44B442EED33919424601A8CD
:1002C00000F05AFFBDF80000BDF80410884202D1CA
:1002D0000120BDE8FC810020FBE70000CD1B0010E1
:1002E000044A02EB401353F8802F8A431A6000F04F
:1002F00023B8000000C00F4000207047FFFFFFFF41
:10030000044A02EB401353F8802F0A431A6000F0AE
:1003100013B8000000C00F4006490122202803D373
:1003200051F8C83F203801E051F8C43F82401343E0
:100330000B60704700C00F40AA21420103481044DF
:1003400040F88C1F552101607047000000C00F402D
:100350000248D0F8040100F01F00704700C00F40B1
:100360000448D0F80401C00501D5012070470020E1
:100370007047000000C00F4000B5FFF7F1FF38B133
:10038000012801D0002000BD5DF804EB00F004B8A6
:100390005DF804EB00F014B8084900B5D1F88820E6
:1003A0000020C2F30022002A07D0D1F8840000F018
:1003B0001F01491C00F004F8484300BD00C00F4075
:1003C0000748D0F80C0110F0030003D0012803D037
:1003D00000207047034870470348006870470000DA
:1003E00000C00F40001BB7009842000000B5FFF7A7
:1003F000C3FF0146FFF7ACFFB1FBF0F000BD42F2D6
:10040000020070474D0B00002DE9F041664C0027BB
:1004100088B0A770E770DFF894814FF40056277119
:1004200001251922314601A800F0A6FE022216215C
:100430003046FFF727FF00287ED0DDF81210022299
:1004400006F11900FFF71EFF002875D09DF8040083
:1004500006282AD2DFE800F02A03032A2A1CD8F84B
:100460007410DDF80E30491C8B421ED2D8F874206F
:10047000DDF80E30D21ADDF81230521C9A4214D335
:10048000DDF80E20DDF812301A448A420DD80DE056
:10049000DDF81210B1F5F42F00D9A570DDF81610B3
:1004A000C1F30B41B1F5407F00D0A570012803D006
:1004B000022801D0052839D1022206F21D416846E2
:1004C000009700F059FE0099029889B2884200D046
:1004D000A570012206F225416846009700F04CFE07
:1004E0000099BDF80500C9B2884200D0A5709DF8FA
:1004F000040002281AD1042206F2494168460097F6
:1005000000F03AFEDDF816000099884200D0A57090
:10051000012206F24D416846009700F02DFE00983A
:100520009DF80710C0B2814200D0A5709DF81C0054
:10053000401EFE2802D200E01EE0A570BDF80500B6
:10054000A0F57F41FF3901D0392802D19DF807007D
:1005500020B901A800F07AFD00B9A570DDF81200FD
:100560001B36064401A800F071FD30B1E07880B17F
:10057000217988420DD012E0A5709DF81C0010B9B9
:100580002079401C2071E078401CC0B2E0700C283B
:1005900001D3A57003E0A07800283FF442AFA07813
:1005A00008B0BDE8F0810000B40000103C4100003C
:1005B000044AD2F8041101F480710143C2F8041115
:1005C0007047000000C00F4006490128D1F804011F
:1005D00005D020F4807000BFC1F80401704740F4DA
:1005E0008070F9E700C00F40044AD2F8B41121F03E
:1005F0001F010143C2F8B4117047000000C00F4052
:100600000449D1F8B42122F4407242EA0020C1F832
:10061000B401704700C00F40044AD2F8081121F01D
:100620001F010143C2F808117047000000C00F40CD
:100630000449D1F8082122F4407242EA0020C1F8AE
:100640000801704700C00F4041EA4211044A02EB22
:100650004012C2F884100121C2F88010FFF76CBE6E
:1006600000C00F4000EB41100121914002680BB126
:100670000A4300E08A4302607047000000F01F0256
:100680004109012090408A0004491144C1F8CC017D
:10069000D1F8CC218243C1F8CC21704700C00F4073
:1006A00010B51D4CD4F8A001C0F3801028B9D4F8BF
:1006B000A00140F02000C4F8A001D4F8A001C0F3CC
:1006C00080100028F9D00020FFF77EFFD4F88800C2
:1006D000C0F3002018B101210020FFF701FE012026
:1006E000C4F80C01002209211046FFF7ADFF0121DB
:1006F0000020FFF705FE0120FFF75AFFD4F888001D
:10070000C0F380200028F9D00120FFF75DFF022010
:10071000C4F8A80110BD000000C00F4010B500F0E3
:1007200011F8BDE81040FFF7F7BD416800224260B4
:1007300001228260022242608268002AFCD141606C
:10074000704700000849884201D1022070470749DC
:10075000884201D1162070470549884201D11720EF
:1007600070470120704700000080004000000940F1
:10077000004009404A0703D5026802F01B020260EC
:10078000090703D5016841F00801016070470021A5
:100790000160FF2141604FF6FF7141616FF07F41C1
:1007A0008161704710B500F011F820B103488068EE
:1007B000BDE81040004742F2020010BD14010010D5
:1007C0000148006800470000140100102DE9F041C5
:1007D0000024012001F010FF9F2000F03BFA00F000
:1007E00021FA60F3070400F01DFA60F30F2400F013
:1007F00019FA60F31744002001F0FEFE234E24484E
:10080000A71B244B244A2549254DB4420FD008DCB0
:10081000A4F1C204B4F5B11419D0B4F5003F13D15A
:1008200015E0204C3C1921D01F4EF4420CD11F4C36
:100830000460C0E903211F49C0E905151E491C4C8D
:10084000C161C0E901431FE00020BDE8F0811B4BFE
:1008500003601B4B43601B4B8360C0E903211A49B3
:1008600041611A4981611A49C1610DE0194C046066
:10087000C0E903211949C0E905151949164CC161A0
:10088000C0E9014301F0FCFC0120DEE7BF25410087
:1008900014010010211C0000D91B0000351D0000B0
:1008A0007123000000FFFEFF0001F8FF051D00009E
:1008B000FD1C00005F1E0000BD1F0000B51A0000F7
:1008C000AD1A0000351A000055170000F917000096
:1008D0002D180000D7210000D1210000DD210000EB
:1008E000A523000012B1024B1B6918470020704776
:1008F0001401001012B1024B9B6918470020704789
:100900001401001038B5049C24B10094024CE46931
:10091000A04738BD002038BD1401001070B509484B
:10092000022400F11F05816829B1007B000607D46D
:10093000022002F09DFB2C7300F0E4FE002070BD4D
:10094000012070BD951B001010B50C480C4C806840
:10095000A178884200D2A0700849A278403982204C
:1009600002F0B4FB032060700448A2781F30816855
:10097000891A81600021017310BD0000951B0010D1
:100980007000001000B572B6064B4FF080509863AF
:10099000002001F031FE4FF0007098674000D867EA
:1009A00000BD00000080092001460007C00E0906B6
:1009B00000D5401C704700002DE9F041092000F0EF
:1009C00051FB154800254FF47A770570C821384649
:1009D000FFF72BFC00F024F8064642F2107400BF2B
:1009E00000F01EF8801BA042FAD3C8213846FFF75A
:1009F0001CFC00F015F8064600F012F8801BA0421F
:100A0000FAD3C8213846FFF710FC0448022185704C
:100A10008171C570BDE8F08168000010B40000105D
:100A20004FF0402080687047FFF7ACFF4FF08044E4
:100A30002046FFF7ACFE43F2D4006060206840F02F
:100A4000020020600C212046FFF794FE206840F051
:100A500001002060AA20A0605520A060FEE70120D0
:100A6000FFF7E2FF0449054A0020C880D064022352
:100A70005360886170470000F00000100080014062
:100A800030B5104B00240AB19A6100E09C610A2243
:100A9000B1FBF2F50C49DD80022285B178B14A60E4
:100AA0000A4AB2FBF0F28A61094AB2FBF0F008642C
:100AB0008814C864012048601120086530BDCC64EA
:100AC0004A6030BDF00000100080014040420F003D
:100AD00020A107002DE9F041354DD5F8C00040F0C8
:100AE0001000C5F8C000334CA08800B972B6A088C9
:100AF000401CA080304908684FF6FF0210402F4A82
:100B00001043086000F0B0F82D494FF00040C1F8E4
:100B10009800FFF76BFC2061D5F8A811072501F0BC
:100B20001F01B0FBF1F161614FF47A71B0FBF1F09C
:100B3000401EB0F1807F09D24FF0E02670611F2186
:100B4000701700F0F4FF0020B06135614FF04026CF
:100B50003046FFF7E3FD3046FFF7E7FD194F6069C8
:100B6000B0FBF7F0401EF060706840F0010070606C
:100B700000F040FA0620FFF7CFFB1348022646603C
:100B80006169B1FBF7F1491EC16046611121016540
:100B90000A20FFF7C1FB0D48066105604660A0888A
:100BA000401E0004000CA08000D162B6BDE8F081B8
:100BB00000C00F40F00000100CED00E00000FA054E
:100BC0000080092040420F000080014000000340E7
:100BD00003484069800401D4012070470020704719
:100BE000008009200348406D400501D40120704772
:100BF000002070470080092003484069C00401D4E8
:100C000001207047002070470080092000B50B4686
:100C1000024603E000F006F802F8010B5B1E9BB2EF
:100C2000F8D200BD044800218160C168C906FCD427
:100C30008068C0B2704700000000034000B50B465A
:100C4000024603E012F8010B00F004F85B1E9BB2B1
:100C5000F8D200BD03498860C868C006FCD4886823
:100C6000C0B270470000034010B5032300221821D2
:100C7000184600F06DFF032300220121052000F03B
:100C800067FF032300220421052000F061FF0323F6
:100C900000221521012000F05BFF00231022072114
:100CA000022000F055FF002380221F21012000F0C8
:100CB0004FFF012300221C21042000F049FF0123E3
:100CC00000221D21042000F043FF032310221946B7
:100CD000052000F03DFF032300220221052000F043
:100CE00037FF012300221321184600F031FF0123B2
:100CF00000220521022000F02BFF032300221C21EB
:100D0000012000F025FF012300221D21184600F0DC
:100D10001FFF002310221721012000F019FF0123DB
:100D200005221821184600F013FF01230522142183
:100D3000184600F00DFF032301220221002000F0DD
:100D400007FF002301220321184600F001FF0222C1
:100D500003230021104600F0FBFE00231222012194
:100D6000022000F0F5FE022203230821104600F0C5
:100D7000EFFE022200230921104600F0E9FE0021C7
:100D800003230222084600F0E3FE00230222012191
:100D9000184600F0DDFE40F202240123224609211C
:100DA000002000F0D5FE00234FF4C1720821184640
:100DB00000F0CEFE012322460721002000F0C8FEED
:100DC000002301221D21184600F0C2FE002301224B
:100DD0001E21184600F0BCFE0123002212211846F5
:100DE00000F0B6FE002380221E21012000F0B0FE9C
:100DF00040F21144032322461C21002000F0A8FEEB
:100E0000032322461B21002000F0A2FE641C0323C2
:100E100022460A21002000F09BFE032322460B21DC
:100E2000002000F095FE002301221946104600F034
:100E30008FFE012200231146104600F089FE012298
:100E400000230421104600F083FE01220023082124
:100E5000104600F07DFE012200230921104600F01B
:100E600077FE012200230A21104600F071FE0122C4
:100E700000230F21104600F06BFE01230022062103
:100E8000022000F065FE032380220E21012000F0E5
:100E90005FFE002381221021012000F059FE002373
:100EA00081221121012000F053FE00230222132190
:100EB000184600F04DFE002302221421184600F0CF
:100EC00047FE002302221521184600F041FE0023B0
:100ED00002221621184600F03BFE022200230B21BD
:100EE000104600F035FE022200230C21104600F0CF
:100EF0002FFE022200230D21104600F029FE0023C0
:100F000010221721032000F023FE012300221621C6
:100F1000184600F01DFE002203230521104600F0B4
:100F200017FE012300221F21042000F011FE0022E1
:100F300003230621104600F00BFE00230122172197
:100F4000184600F005FE002301221821184600F083
:100F5000FFFD002301221921184600F0F9FD0023AE
:100F600001221A21184600F0F3FD03230022192163
:100F7000184600F0EDFD012300221A21032000F0A5
:100F8000E7FD01231A460321022000F0E1FD0123C1
:100F900000221A21184600F0DBFD002310221B213D
:100FA000012000F0D5FD002390220D21184600F00D
:100FB000CFFD002310220A21022000F0C9FD0023EA
:100FC00090220C21184600F0C3FD022103230022C9
:100FD000084600F0BDFD032300220421022000F09A
:100FE000B7FD00220123BDE810400E21104600F09D
:100FF000AFBD000070B5134C2046FFF78FFB2046B5
:10100000FFF793FB606940F0080060610E486421BF
:101010004069B0FBF1F0211D401E88616069042524
:1010200040F010006061606840F0010060604FF0C7
:10103000E024C4F880520E210220843400F077FDB1
:10104000E56770BD00800040F00000100021425CA8
:1010500012B9491C1829FAD3182901D00020704769
:10106000012070472DE9F041374C88B12246042514
:10107000D268D4F808C093060226EF053349521C03
:10108000BCF1050F07D2DFE80CF008172642580024
:101090000020A060E060BDE8F081042849D0052868
:1010A00045D0012502284BD0012838D001E0A560A9
:1010B000F1E70E2844D0EEE7062808D00328EAD04E
:1010C000092836D00D2810D00C2832D0E3E700F0E4
:1010D0003FF8A660DFE706280BD00A2812D00928BF
:1010E0001DD00C2825D00D28D5D1BDE8F04100F049
:1010F0002FB84FF08060E260002B01DA8867CAE702
:10110000C867C8E700F02EF80320A060C3E70728EF
:1011100008D00A280DD00B2812D00928BBD100F026
:1011200021F8C4E7E260002B01DA8F67B3E7CF67ED
:10113000B1E7BDE8F04100F015B80628C7D0B8E720
:1011400000F006F8B3E70000F0000010008009206E
:1011500003484FF00071C167490081677047000084
:101160000080092003484FF0007181674900C16782
:10117000704700000080092010B50B46014600248E
:101180001846FFF7AFFB204610BD00000E4810B513
:101190004178022908D003290ED0042910D005294E
:1011A00001D10021417010BD0848C07B2828FAD128
:1011B000BDE8104000F034B9BDE8104000F0A2BA1C
:1011C000822001F055FFF7E770000010951B00101A
:1011D00010B51449022001F055FD13498870487874
:1011E00060B101280ED0022001F042FF0D4902201B
:1011F0005F310873BDE8104000F084BABDE81040CC
:1012000000F014B807484030C07B2A2805D02F28AA
:1012100007D1BDE8104000F035B9BDE8104000F03E
:1012200075B910BD551B0010700000102DE9F0417C
:101230004A4D4B4C0021A878A4F1400202E0535CD7
:101240006354491C03468142F9D31F2B7CD120688B
:101250004449884278D1424E60681F364FF00108F9
:101260007060A068B060607B18B9A07B08B11028DE
:1012700002D986F80C8063E0E07B1E28F9D011DCEF
:10128000122833D006DC68B30328F2D1BDE8F04160
:1012900000F00EBA1528ECD01A28EAD1BDE8F041CA
:1012A00000F07EB902272A282ED011DC232821D075
:1012B000252823D02828DCD100F08AF900282CD05A
:1012C000207B00061ED56F70BDE8F04100F0A8B885
:1012D0002F2824D05528CCD05A28CAD1BDE8F041B7
:1012E00000F042B9BDE8F04100F01EBABDE8F0419F
:1012F00000F03AB8BDE8F04100F0B4B9BDE8F04103
:1013000000F08EB9022018E000F062F9002804D045
:10131000207B000610D485F80180BDE8F08100F044
:1013200057F90028F9D0207B000605D485F8018004
:10133000C5F82880F1E707E0822001F099FE3773B5
:10134000BDE8F04100F0DEB9822001F091FE0220FC
:1013500001F08EFE06206870DFE7000070000010CC
:10136000951B0010555342431CB5FFF7D7FA0028D0
:101370004ED028480A2206210388684602F000FC65
:101380002548002280230270437082700121C170C1
:101390002021017143718271C27141220272542273
:1013A00042724F2282724C22C27201734173817366
:1013B000C1734622027450234374722383746923D9
:1013C000C3746E230375742343758175C2756C22D3
:1013D000027661224276732282766822C276017793
:1013E00041778177C1779DF8011080F820109DF832
:1013F000021080F821109DF8031080F822109DF84B
:10140000041080F82310054924208870FFF79CFA07
:101410001CBD000004040000551B001070000010EB
:1014200070B5154D2C6B402C00D94024E86AE96951
:1014300002198A4202D90C1A04216970214602F06D
:10144000E7FA22460D49822001F040FEE86A204476
:10145000E862286B011B0A4829638268A2EB040238
:10146000826005D06978022901D00021017370BD26
:1014700003216970F9E7000070000010CD1B001017
:10148000B41B00102DE9F0411D4CA178E06A421810
:10149000E1698A4206D9081AA0700520607002200E
:1014A00001F0E6FD0021A078164B174DE26A08E036
:1014B00056186F5C9E5DBE4202D00021A16202E020
:1014C000491C8142F4D31118E162216B0A1A0E49BA
:1014D000226301F15F018B68A3EB0000886002D0FA
:1014E0006078052809D1A06A28B100200873BDE8FA
:1014F000F04100F007B90120F8E7BDE8F0810000F5
:1015000070000010CD1B0010551B001010B5144CBE
:10151000A178E06A4218E1698A4206D9081AA070E7
:1015200005206070022001F0A3FDA178E06A02F0BE
:10153000B5FAA178E06A0844E062206B421A0948D3
:1015400022638368A3EB0101816002D061780529E1
:1015500005D100210173BDE8104000F0D3B810BDE3
:1015600070000010B41B001010B5FFF7D7F9002869
:1015700011D0094800210622017042708170C170AB
:10158000017141718171C171044908208870BDE801
:101590001040FFF7D9B910BD551B001070000010A6
:1015A00010B5FFF7BBF900280DD0074803210170E3
:1015B000002141708170C170044904208870BDE829
:1015C0001040FFF7C1B910BD551B0010700000108E
:1015D000114810B5D0F81110027D09BA21F0FF01B1
:1015E00011430E4A4902D162C18A49BA49021163C4
:1015F000806888420DD0822001F03AFD022001F07F
:1016000037FD054902201F31087300F07BF80020E8
:1016100010BD012010BD0000951B001070000010CF
:1016200010B5FFF77BF9002816D00C4A0C48116A58
:10163000491E0B0E03700B0C43700B0A8370C170B4
:1016400000210171417102238371C17108209070E2
:10165000BDE81040FFF778B910BD00007000001021
:10166000551B001010B5FFF759F900281AD00E4885
:1016700000210E4B0170417081700822C2701A6AFD
:10168000140E0471140C4471140A8471C271022284
:10169000027241728272C1720C209870BDE81040D3
:1016A000FFF752B910BD0000551B0010700000106C
:1016B00010B5FFF733F900281FD01048702102221F
:1016C0000170002141708270C1700171417181719E
:1016D0000A22C271017241728172C1723022027398
:1016E000012242738173C173017441740449122051
:1016F0008870BDE81040FFF727B910BD551B0010DA
:1017000070000010064910B5044808600D228220C0
:1017100001F0DCFC03490520487010BD55534253CD
:10172000B41B001070000010094810B5816839B171
:10173000007B000601D5822000E0022001F098FC29
:10174000034900201F310873BDE81040FFF7DABFDE
:10175000951B00102DE9FC5F5FEA02084FF00006C0
:101760008A4624D04FF4805501462A466846FEF743
:10177000D9FCDDE90047284602F0D6F85FEA000907
:1017800017D0AB46A8EB0605C7F58050A84200D29B
:1017900005465D4510D02046494600F005FB58B18E
:1017A000484602F047F842F20400BDE8FC9F0020E2
:1017B000FBE742F20100F8E7204600F077FA60B953
:1017C0000AEB060107EB09002A46FEF7B5FC2E449A
:1017D0002046494600F0E4F828B1484602F02AF8CD
:1017E00042F20500E1E70027641C4645CAD348469B
:1017F00002F020F8DBE700002DE9F04117008046F9
:101800000D460DD00024084E08E0295D08EB0400C9
:1018100000F05EFD3060002803D1641CBC42F4D3AC
:101820000020BDE8F08100006C0000102DE9FF4FA2
:101830008FB00C46DDF87080002608935FEA08013F
:1018400077D04FF4805501462A466846FEF76AFC79
:10185000DDE900A10D912A46611C6846FEF762FC95
:10186000DDE900B104912A4668461199FEF75AFC59
:10187000DDE90045A8EB0607C5F58050B84200D267
:10188000074625B1544573D10D98854270D14FF468
:10189000805002F049F85FEA00090BD0544535D179
:1018A0000D98854232D12A462003494600F04EFA6F
:1018B000F0BB04E042F2010013B0BDE8F08F5C45DC
:1018C00009D104990498C1F5805200EB0B304944CA
:1018D00000F03CFA60BB204600F0E8F940BB0898F5
:1018E0003A46811905EB0900FEF726FCEA192003A8
:1018F000494600F03DFDD8B95C4535D104990498BE
:10190000C1F5805200EB0B30494423E05C4509D11E
:1019100004990498C1F5805200EB0B30494600F061
:1019200015FA28B9204600F0C1F908B9089801E075
:1019300013E030E0811911983A46304400F018FD68
:1019400058B95C4510D104990498C1F5805200EB58
:101950000B30494600F00CFD30B1484601F06AFFFB
:1019600042F20500A8E703E0484601F063FF0CE0FF
:1019700008983A4681191198304400F0F9FC07495B
:10198000086010B10846006896E73E440025641CD4
:101990004645FFF46FAF00208EE700006C0000109A
:1019A0002DE9F04FC3B00024DFF884B08A46054625
:1019B000A0466F464FF00209C0F3071641A95846EA
:1019C00000F038FA50BB9DF80401800701D400F004
:1019D000CFFA8DF800908DF8016004EB05108DF8BA
:1019E00002008DF803800AEB04214FF48072381D49
:1019F000FEF7A2FB012000F0FFFD4FF48271684664
:101A0000FFF71CF9002000F0F7FD641CE4B2102C75
:101A1000D4D341A9584600F00DFA20B142F2050096
:101A200043B0BDE8F08F00F097FA0020F8E700001F
:101A3000A08601002DE9F0410026012000F0DCFD28
:101A40009F20FFF707F9FFF7EDF80746FFF7EAF8E1
:101A50000546FFF7E7F80446002000F0CDFDC22F51
:101A600001D1202D03D042F20200BDE8F0810E49E1
:101A7000142C0BD0152C0CD0162C0ED0182C0FD0EB
:101A80000E60002000F01CF80020EEE74FF48010FC
:101A900001E04FF400100860F3E74FF48000FAE72C
:101AA0004FF08070F7E700000C0100104FF48050F9
:101AB0007047000001480068704700000C010010EA
:101AC00070B5184C05464FF080762068B0420BD1B7
:101AD000012000F091FD1520FFF7BCF83846FFF714
:101AE000B9F8002000F088FD012000F085FD0620F7
:101AF000FFF7B0F8002000F07FFD012000F07CFD32
:101B00000120FFF7A7F8A806000EFFF7A3F820684A
:101B1000B04202D13846FFF79DF8BDE87040002082
:101B200000F06ABD0C0100100120FEF77DFFC90620
:101B3000090E002806DA00F00F0000F1E02080F81E
:101B4000141D704700F1E02080F800147047000079
:101B500070B504460E480D4600EBC4101E4640F812
:101B600025200C48D90701D0012300E000232A4694
:101B70002146FEF777FD074BB2074FF0010000FA50
:101B800005F003EB441101D5886170BDC86170BDDB
:101B900000C002400080092010B5FEF703FEFEF7EA
:101BA0000FFE04494FF40052C1E90020A0F5F420D3
:101BB000886010BDA800001006493022C1F8082234
:101BC000C1F81002D1F800028006FBD5D1F814024A
:101BD0007047000000C0082038B569460E4800F084
:101BE00029F942F20504A0B99DF80000800701D44C
:101BF00000F0BEF9012000F0FFFC6020FFF72AF89A
:101C0000002000F0F9FC6946044800F013F90028B0
:101C100000D0204638BD0000A086010020A10700AA
:101C20002DE9F0410026012000F0E6FC9F20FFF79F
:101C300011F8FEF7F7FF0746FEF7F4FF0446FEF73C
:101C4000F1FF0546002000F0D7FCBF2F02D0C22FC5
:101C500005D006E0252C08D0262C06D001E0202C4B
:101C600003D042F20200BDE8F0810F48412D14D0AC
:101C700004DC142D0ED0182D06D112E04FF4800193
:101C8000422D0CD04A2D0AD00660002000F0B8F892
:101C90000020E8E74FF4801101E04FF400110160EB
:101CA000F3E74FF08071FAE71001001038B50446F1
:101CB0006946114800F0BEF810B142F2050038BD87
:101CC0009DF80000800701D400F052F9012000F0D7
:101CD00093FC2020FEF7BEFFC4F30710FEF7BAFF07
:101CE0002007000EFEF7B6FF0020FEF7B3FF00202E
:101CF00000F082FC002038BDA08601004FF4805027
:101D00007047000001480068704700001001001093
:101D100010B50446012000F06FFC0520FEF79AFF85
:101D2000FEF780FF2070002000F066FC207800F0B5
:101D3000010010BD10B522B100F008F8024908609A
:101D400010BD002010BD00006C000010F8B515009B
:101D50000E46044607D06946124800F06BF820B1E1
:101D600042F20400F8BD0020F8BD012000F044FC60
:101D70000B20FEF76FFFC4F30740FEF76BFFC4F3C1
:101D80000720FEF767FFE0B2FEF764FF0020FEF7D2
:101D900061FFA9B23046FEF739FF002000F02CFCAD
:101DA000E1E70000A086010038B50D46044669460B
:101DB000124800F03FF810B142F2040038BD012093
:101DC00000F01AFC0B20FEF745FFC4F30710FEF7E6
:101DD00041FF2007000EFEF73DFF0020FEF73AFF0F
:101DE0000020FEF737FF4FF480512846FEF70EFF24
:101DF000002000F001FC002038BD0000A08601009A
:101E000010B50446012000F0F7FB5020FEF722FF3A
:101E1000002000F0F1FB012000F0EEFB0120FEF7B6
:101E200019FFA006000EFEF715FFBDE810400020C8
:101E300000F0E2BB70B50E460546FEF7F1FD044624
:101E400007E000BFFEF7ECFD001BA84201D3012014
:101E500070BD3046FFF75CFF0028F3D170BD2DE95F
:101E6000FC5F5FEA02084FF000068A4624D04FF478
:101E7000805501462A466846FEF754F9DDE90047D9
:101E8000284601F051FD5FEA000917D0AB46A8EBE8
:101E90000605C7F58050A84200D205465D4510D022
:101EA00020464946FFF780FF58B1484601F0C2FC82
:101EB00042F20400BDE8FC9F0020FBE742F2010073
:101EC000F8E72046FFF7F2FE60B90AEB060107EBE0
:101ED00009002A46FEF730F92E442046494600F014
:101EE00025F928B1484601F0A5FC42F20500E1E7DA
:101EF0000027641C4645CAD3484601F09BFCDBE73B
:101F000038B50D46044669461248FFF793FF10B1F5
:101F100042F2050038BD9DF80000800701D400F0B2
:101F200027F8012000F068FB0220FEF793FEC4F3BF
:101F30000740FEF78FFEC4F30720FEF78BFEE0B2EA
:101F4000FEF788FE2846FEF785FE002000F054FBD1
:101F5000002038BDA086010010B5012000F04CFB28
:101F60000420FEF777FEBDE81040002000F044BBDF
:101F700010B5012000F040FB0620FEF76BFEBDE827
:101F80001040002000F038BB2DE9F04117008046DA
:101F90000D460DD00024084E08E0295D08EB040032
:101FA000FFF7AEFF3060002803D1641CBC42F4D3BD
:101FB0000020BDE8F08100006C0000102DE9FF4F0B
:101FC0008FB00C46DDF87080002608935FEA0801A8
:101FD00077D04FF4805501462A466846FEF7A2F8AE
:101FE000DDE900A10D912A46611C6846FEF79AF8CA
:101FF000DDE900B104912A4668461199FEF792F88E
:10200000DDE90045A8EB0607C5F58050B84200D2CF
:10201000074625B1544571D10D9885426ED14FF4D4
:10202000805001F081FC5FEA00090BD0544535D1A6
:102030000D98854232D12A4620034946FFF786FE95
:10204000F0BB04E042F2050013B0BDE8F08F5C4540
:1020500009D104990498C1F5805200EB0B30494432
:10206000FFF774FE60BB2046FFF720FE40BB0898D8
:102070003A46811905EB0900FEF75EF8EA192003DC
:102080004946FFF781FFD8B95C4532D104990498DD
:10209000C1F5805200EB0B30494423E05C4509D187
:1020A00004990498C1F5805200EB0B304946FFF7C4
:1020B0004DFE28B92046FFF7F9FD08B9089801E060
:1020C00013E02EE0811911983A463044FFF75CFF87
:1020D00058B95C450DD104990498C1F5805200EBC4
:1020E0000B304946FFF750FF18B1484601F0A2FBFC
:1020F000A8E7484601F09EFB0DE0FFE708983A4646
:10210000811911983044FFF73FFF0749086010B16B
:102110000846006898E73E440025641C4645FFF4E5
:1021200071AF002090E700006C0000102DE9F8432B
:10213000264E0D46044669463046FFF77BFE42F2C6
:102140000507D8BB9DF80000800701D4FFF710FFFA
:10215000012000F051FAAD20FEF77CFDC4F307101A
:10216000FEF778FD2007000EFEF774FD0020FEF755
:1021700071FD02212846FEF761FD002000F03CFAC7
:102180000224B046E60269464046FFF753FEA8B96E
:10219000012000F031FAAD20FEF75CFD2819022184
:1021A000FEF74CFD002000F027FAA41CA4B2B442B4
:1021B000E9D369464046FFF73DFE10B13846BDE819
:1021C000F883FFF7C9FE0020F9E70000A0860100B0
:1021D0004FF4805070474FF4800070472DE9FC5F4A
:1021E0005FEA02084FF000068A4624D04FF480557B
:1021F00001462A466846FDF795FFDDE90047284677
:1022000001F092FB5FEA000917D0AB46A8EB060588
:10221000C7F58050A84200D205465D4510D0204643
:102220004946FFF7C1FD58B1484601F003FB42F2B1
:102230000400BDE8FC9F0020FBE742F20100F8E744
:102240002046FFF733FD60B90AEB060107EB0900F2
:102250002A46FDF771FF2E442046494600F05CF9FE
:1022600028B1484601F0E6FA42F20500E1E700270E
:10227000641C4645CAD3484601F0DCFADBE700009F
:102280001FB503A91148FFF7D5FD18B142F20500AB
:1022900004B010BD9DF80C00800701D4FFF768FE64
:1022A00042208DF800000020CDF80100CDF8050097
:1022B000ADF80900012000F09FF90B216846FEF7F8
:1022C000BDFC002000F098F90020E1E7A0860100A5
:1022D0002DE9FF41254F0D46044669463846FFF774
:1022E000A9FD42F20506F0B99DF80000800701D46F
:1022F000FFF73EFE42208DF804000020CDF80500D7
:10230000CDF80900ADF80D00012000F075F90B21A2
:1023100001A8FEF793FC002000F06EF969463846EC
:10232000FFF788FD18B1304604B0BDE8F0819DF894
:102330000000800701D4FFF71BFE02208DF8040087
:10234000200C8DF80500200A8DF806008DF8074056
:102350008DF80850012000F04FF9052101A8FEF783
:102360006DFC002000F048F90020DDE7A0860100A8
:102370002DE9F041170080460D460DD00024084E8F
:1023800008E0295D08EB0400FFF7A2FF3060002899
:1023900003D1641CBC42F4D30020BDE8F0810000EE
:1023A0006C0000102DE9FF4F8FB00C46DDF87080F7
:1023B000002608935FEA080177D04FF48055014664
:1023C0002A466846FDF7AEFEDDE900A10D912A46DA
:1023D000611C6846FDF7A6FEDDE900B104912A46BE
:1023E00068461199FDF79EFEDDE90045A8EB06075A
:1023F000C5F58050B84200D2074625B1544573D187
:102400000D98854270D14FF4805001F08DFA5FEA4B
:1024100000090BD0544535D10D98854232D12A465A
:1024200020034946FFF792FCF0BB04E042F20100B2
:1024300013B0BDE8F08F5C4509D104990498C1F54B
:10244000805200EB0B304944FFF780FC60BB204614
:10245000FFF72CFC40BB08983A46811905EB0900B0
:10246000FDF76AFEEA1920034946FFF781FFD8B954
:102470005C4535D104990498C1F5805200EB0B30CE
:10248000494423E05C4509D104990498C1F5805280
:1024900000EB0B304946FFF759FC28B92046FFF7FF
:1024A00005FC08B9089801E013E030E081191198A3
:1024B0003A463044FFF75CFF58B95C4510D10499A7
:1024C0000498C1F5805200EB0B304946FFF750FFEE
:1024D00030B1484601F0AEF942F20500A8E703E04A
:1024E000484601F0A7F90CE008983A46811911987E
:1024F0003044FFF73DFF0749086010B10846006807
:1025000096E73E440025641C4645FFF46FAF00206B
:102510008EE700006C0000102DE9F04FC3B00024DE
:10252000DFF884B08A460546A0466F464FF00209A0
:10253000C0F3071641A95846FFF77CFC50BB9DF835
:102540000401800701D4FFF713FD8DF800908DF88A
:10255000016004EB05108DF802008DF803800AEB92
:1025600004214FF48072381DFDF7E6FD012000F0D4
:1025700043F84FF482716846FEF760FB002000F0DC
:102580003BF8641CE4B2102CD4D341A95846FFF7A1
:1025900051FC20B142F2050043B0BDE8F08FFFF7D7
:1025A000DBFC0020F8E70000A0860100F8B5144627
:1025B000074E0A460B19716800258B4200D90A1B89
:1025C000034600943068FEF79DF92846F8BD0000E8
:1025D000A800001070B5034608468D180549002470
:1025E00049688D4200D9881A1946FEF783F92046BA
:1025F00070BD0000A80000104021034A012801D04E
:1026000091617047D16170470080092070B5054D18
:102610004FF48004012803D0FEF7B4F9AC63FEE761
:10262000EC6370BD00800920054910B50878421C94
:102630000A700A2803D30020087000F025F810BDA6
:10264000F00000100D4810B50D4901602020FEF784
:1026500015F80C480321C0F8B0110168C1F30B0153
:1026600041F440510160FEF71BF80220FDF7BCFF6A
:10267000BDE810400120FDF7C3BF000008ED00E0F9
:102680000000000000C00F400748C188002909D0A1
:10269000491E0904090CC18004D1806900B10047BA
:1026A000FEF7E0B970470000F0000010154810B5C3
:1026B0000168016014494878C82801D2401C48705C
:1026C000FEF786FA00220028C8780CD030B148788E
:1026D000322800D98A700120C87010BD8878401C4B
:1026E00088704A70F7E708B14A7003E048783228EA
:1026F00000D98A70CA7088780328EED10020FFF7CD
:1027000085FF10BD00800040F000001000B5FEF70E
:102710004BF904495DF804EB41EA0040891300F0ED
:1027200017BD00000005400010B502468078FEF796
:102730003BF90B49D1F84432012484402343C1F8CA
:102740004432C1F848029088C1F84C02D1F8000226
:10275000C005FBD54FF48070C1F8080210BD000021
:1027600000C0082010B500B101204FF4807444EA85
:102770000041074800F0ECFC06480321C0F8441271
:10278000D0F80012C905FBD5C0F8084210BD000002
:102790000005D80000C008207047000010B50400F4
:1027A00001D0012000E000204FF4807141EA004197
:1027B000054800F0CDFC05494FF480200CB188633A
:1027C00010BDC86310BD00000005FE000080092098
:1027D00010B5084CA288402A00D9402280202168E8
:1027E00000F074FC216801442160A188081AA080CF
:1027F00010BD0000D800001010B5064C0020216864
:1028000000F040FA216801442160A188081AA080E4
:1028100010BD0000D80000107047000000B5FEF7A2
:10282000C3F804495DF804EB41EA0040024900F0B6
:102830008FBC0000000540000001200000B5FEF73D
:10284000B3F804495DF804EB41EA0040891300F055
:102850007FBC0000000540002DE9F0414A4C0027F4
:10286000A4F108062178A4F11C05082864D2DFE849
:1028700000F0630465746363868400F009FC2078CB
:10288000C009FFF7C9FFE088B0802078C0F341118C
:10289000F1BB61780C294BD2DFE801F006094A0B45
:1028A0004A101B1E2026324300F0B6F84EE00020EE
:1028B00000E0012000F074FA50B306E010F01F0FA2
:1028C00036D1A07840F080002870BDE8F04100F0DB
:1028D000E5BB00F065F839E000202AE010F01F0F9A
:1028E00026D129481B381AE010F01F0F20D100F024
:1028F0009FFA68B100F0D2FBBDE8F041FFF74CBF92
:1029000000F01F00012813D1687808B1207900E099
:102910000EE0A97888420BD21B490C39084430607C
:102920001DE000F01F00012802D100F029FBC3E7E1
:10293000802000F09DFBB780BDE8F081080608D438
:10294000B0880028F8D0FFF757FFB0880028EFD0F4
:10295000F2E7BDE8F04100F0A7BB080603D5BDE8EB
:10296000F041FFF735BF28780106E5D500F07F007C
:102970002870BDE8F04100F0FFB9802000E00020A1
:10298000BDE8F041FFF7C2BEE0000010022803D00E
:10299000032803D1FEF7FABBFEF71ABC704700000C
:1029A000194810B5007810F01F0F1748C07829D1CA
:1029B00015490839012806D0134A0228937806D011
:1029C00003281FD112E011480860122012E01048BD
:1029D000002204E004780CB144882044521C934245
:1029E000F8D1027872B10860408803E009481844C1
:1029F000086000788A88824200D98880FFF7E8FE64
:102A0000012010BD002010BDE0000010B441000006
:102A1000C6410000E741000070B51D481C4D00781C
:102A2000A5F1080510F01F040AD01948A5F11401FA
:102A3000184B4A780079012C06D0022C26D109E0E7
:102A40001348183828601DE002B3897888421DD2E7
:102A5000002015E000F08F04200605D504F00F06D5
:102A60004FF48030B04001E00120A0400AB92207B5
:102A70000CD18A68024209D0C9680142E8D001201D
:102A800018802B60FFF7A4FE012070BD002070BDF0
:102A9000E0000010381D00102DE9F0412F4DD5F851
:102AA0000032C5F80832180721D52D4800F042FB46
:102AB0002C48FFF781F8C10605D500F019F9BDE8EB
:102AC000F04100F04DB9810705D5BDE8F04100F0B7
:102AD000010000F091B8010709D5400703D5BDE812
:102AE000F04100F0E7BABDE8F04100F043B91E4EF6
:102AF00058074FF001071DD4BDE8F0815FF00004D6
:102B0000D5F8302207FA04F10A4210D06008C5F85F
:102B1000381200BFD5F800128906FBD5D5F814127B
:102B2000E2070CD056F8201009B103208847641C36
:102B3000202CE5D3D5F830020028DFD1DCE73CB902
:102B4000490705D5316819B1012088470124D7E725
:102B500056F820100029EAD00220E7E700C008203C
:102B60000005FE000002FE00584200001F4810B59C
:102B7000D0F8A800C0F3002018B101210846FDF7E5
:102B8000AFFB002207210120FDF75EFD0121084671
:102B9000FDF7B6FB1548202410F12000D0F888106E
:102BA0004905FBD50220FDF737FD0220FDF740FD6A
:102BB0001F20FDF7B1FB0E4912200860091D0A68AD
:102BC00030EA0202FBD14FF0E0214FF08070C1F8F3
:102BD0008002084A82F80044C1F8000100F088F839
:102BE000BDE81040002000F0C7B8000000C00F4052
:102BF000F4CF082018E000E0002802D101490120AC
:102C000048707047E800001070B51A4C607830B317
:102C10000025012811D002280ED1FDF701FF6168BF
:102C2000401A1549884217D31448406B400013D509
:102C30000120FFF7B3FD657070BDFDF7F1FE61681F
:102C4000401A0F498842F7D30020FFF7A7FDFDF790
:102C5000E7FE60600220607025700C2005E020789F
:102C60000028E9D1012020700D20BDE87040FEF75A
:102C7000F9B90000E8000010A086010000800920DA
:102C800040420F0000F00F02012370B503EB8203F6
:102C9000154AC2F8283200BFD2F820321C05FBD5F5
:102CA000C3F309030024DD1C05E000BFD2F818625D
:102CB00041F8046B641CB4EB950FF7D30021C2F804
:102CC000281241F24821C140C9070AD1FDF76CFE24
:102CD0004FF4A06141EA004000F02CFA034800F0F4
:102CE00029FA184670BD000000C008200005F20057
:102CF0000D480021C0F848124021C0F84C120122B2
:102D0000C0F84822C0F84C12D0F80012C905FBD513
:102D10004FF0FF31C0F83812C0F83412C0F8081272
:102D20000C21C0F80412704700C00820044800219C
:102D30004FF00112818001704170C0E9022170479B
:102D4000C400001000B5FDF72FFE04495DF804EB48
:102D500041EA0040891300F0FBB900000005400083
:102D600010B5FFF7E3FF02490020487010BD0000D6
:102D7000E80000107047000030B50749074D41EAF0
:102D800000442146284600F0E3F921462846BDE8E4
:102D9000304000F0DDB90000000180000005D000E7
:102DA00070B502462148A0F11C04017811F01F0300
:102DB0000146498804D0012B29D0022B27D111E0EC
:102DC000012924D132B1012000F07EF9A08840F021
:102DD000020005E0002000F077F9A08820F0020052
:102DE000A08021E0007900F08F00030605D500F0F7
:102DF0000F034FF480359D4001E001258540637845
:102E00002BB1030703D0A3682B4200D009B10020E7
:102E100070BD22B100F02CF9E068284303E0FFF711
:102E200075FCE068A843E060012070BDE000001080
:102E30002DE9F84F504F00200090B8784FF000096E
:102E40004FF0010A4FF4803BA7F11C0600286AD01E
:102E50004A4C64E06078022804D0042840D0052859
:102E60005BD140E06179B878814237D170702079C8
:102E7000B070414900200C3901F80090401C042832
:102E8000FAD301254FEA06080AFA05F0D8F8081027
:102E9000084202D02846FFF7C1FCD8F808100BFA08
:102EA00005F0084203D045F08000FFF7B7FC6D1C29
:102EB000102DE9D34FF00110C8E902090120FFF7F6
:102EC00051FCE0794006B8F8040002D540F001005A
:102ED00001E020F00100A8F804001EE060881DE079
:102EE000E078009019E00098B8B9A07800F08F055C
:102EF000280604D505F00F010BFA01F001E00AFAEB
:102F000005F0B16801432046B160FFF70DFC28468B
:102F1000FFF794FC2846FFF715FF2078044420783B
:102F2000002897D11FE086F8019001245546D84625
:102F3000B16805FA04F0084202D02046FFF76EFCA3
:102F4000B16808FA04F0084203D044F08000FFF7AB
:102F500065FC641C102CEBD34FF00110C6E902098C
:102F60000020FFF7FFFBB8787178884202D101207A
:102F7000BDE8F88F0020FBE7E0000010C64100002C
:102F80002DE9FC5F384D00273E466878BB46B846C1
:102F9000002866D0BA46354C05F11C095DE0607822
:102FA000022804D0042808D0052854D119E06079FB
:102FB000697888424FD060884EE0A77899F804106D
:102FC000E6784FF00008B94245D199F80200B042C6
:102FD00041D125484FF0010A103010F807B0C6550E
:102FE00039E099F80410B94235D1A17801F08F0188
:102FF0000191090605D5019901F00F024FF48031C6
:1030000001E0019A01219140009199F80200B0423B
:1030100013D1A8680843A860E96800988143204656
:10302000E960FFF781FB0198FFF708FC0198FFF7C3
:1030300089FE009948EA01080DE05E450BD118EAC7
:10304000010F08D1A8688843A860E8688843E86051
:103050000198FFF7E3FB20780444207800289ED1F4
:103060005046BDE8FC9F0000C4000010C6410000AF
:1030700000B5FDF799FC04495DF804EB41EA004016
:10308000024900F065B800000005400000010100A1
:1030900001490020FFF7F6BDE000001000221146B4
:1030A000802000F013B8000001490020FFF7EABDBE
:1030B000381D001010B5034C01206070FDF7B0FC06
:1030C000606010BDE80000107047000070B5134646
:1030D0000546134C00F00F00022202EB8000C4F8FA
:1030E0002802C4F824320020DA1C04E051F8046BF2
:1030F000C4F81C62401CB0EB920FF7D30020C4F858
:1031000028022846FDF750FC4FF4A06141EA004038
:1031100000F010F8034800F00DF8184670BD0000EC
:1031200000C008200005FA000420FDF77DFC1020F7
:10313000FDF77AFC05491022C1F80822C1F81002F7
:10314000D1F80002C006FBD57047000000C008207F
:10315000094A1023C2F80832C2F81002D2F800025D
:10316000C006FBD5C2F80832C2F81012D2F800022D
:10317000C006FBD57047000000C008200FB41CB586
:103180000A46521ECDE9000207A9054B6A46069879
:1031900000F018F8009A002111701CBC5DF814FBB7
:1031A0007D33000002E008C8121F08C1002AFAD1CE
:1031B00070477047002001E001C1121F002AFBD1B7
:1031C000704700002DE9FF4F8BB09A460F46054629
:1031D000002606E025280BD052460D9990476D1C1D
:1031E000761C28780028F5D10FB03046BDE8F08F66
:1031F0000024A0460122604900E0044315F8013F85
:10320000203B02FA03F00842F7D128782E2817D184
:1032100015F8010F44F004042A280ED06FF02F0295
:103220002878A0F1300109290AD808EB880102EBBF
:10323000410100EB01086D1CF2E757F8048B6D1C8F
:10324000287869283ED006DC0028CDD063280BD032
:10325000642804D136E0732810D075284BD052462C
:103260000D999047761C85E017F8040B8DF8000047
:1032700000208DF80100E946012003E057F8049B87
:103280004FF0FF3061074FF0000401D40AE0641CE6
:1032900044450DDA8442FADB19F804100029F6D10E
:1032A00006E0641C8442FCDB19F804100029F8D104
:1032B000264404E019F8010B52460D999047641E0C
:1032C000F8D257E001CF4FF00A0B002802DA404253
:1032D0002D2102E0210504D52B218DF82410012198
:1032E00003E0E10705D02021F7E70DF1200908915F
:1032F0000CE00021F9E701CF4FF00A0BF9E759463E
:10330000FCF72CFF01F1300209F8012D0028F6D15D
:10331000ADEB090000F1200B600701D44FF001086C
:10332000D84502DDA8EB0B0000E000208046002419
:1033300006E009A85246005D0D999047641C761C72
:1033400008988442F5DB04E0302052460D999047FE
:10335000761CB8F10001A8F10108F5DC05E019F8C8
:10336000010B52460D999047761CBBF10001ABF161
:10337000010BF4DC6D1C34E7092801004A68002ABF
:1033800006D00A68531C0B6010704868401E4860E5
:103390007047000070B5FDF72FFC78B1FDF740FBDA
:1033A000044643F6982500BFFDF73AFB001BA842F0
:1033B000FAD3FDF721FC08B1012070BD0520FDF70F
:1033C00051FE002070BD0000F0B505460020034608
:1033D00002462B4C4FF4007700E05B1CEE5C46B1DC
:1033E00002EB030CA4440CF5805C9CF800C8B445C7
:1033F000F3D0032B3FD302F5C0502044037F457F19
:10340000C67F03EB0523857F2D0405EB06652B4462
:1034100051EA03052BD021B91A49496840318B4242
:1034200025D8194B00215518254405F5805595F8E8
:1034300000585D54491C0C29F5D3817EC27E01EBF6
:103440000221027D407D120402EB00600C18204630
:1034500000F0A0FA40F6F57502E000BF00F09AFA1D
:10346000C11EA942FAD3A0F57061FF3901D0002036
:10347000F0BD2046F0BD2032BA42AFD3F0BD00000F
:103480005501001070000010C11B00108AB04620CA
:103490008DF818004FF000093920CA4600905446B4
:1034A0008DF81B90AFA3B0A20A2106A8FFF766FE15
:1034B000AF4908684FF6FF021040AE4A40F48070F2
:1034C00010430860AC48AE49B14B0460AB48B14C06
:1034D0000068A0F56C50FF380860AA4900F5E0507C
:1034E0000860A949400A0860A849F8200870FF2030
:1034F0004870887094F90520002053F822200B189A
:1035000003F58053155C401C83F800586028F6D3FF
:103510004FF4E175294640F24910FCF786FE294632
:1035200040F29F10FCF781FE4FF4005BDFF86882E9
:103530005D46207808B1FFF767FBA07928B1012824
:1035400019D0207800286ED0FCE00A20FDF78AFD13
:10355000FCF75AFF18B100BFFDF72EFAE9E701208A
:10356000A0715D4684F803A00620FDF77BFD0A20CC
:10357000FDF778FDDDE7192229468748FDF7FCFDB8
:1035800098F8180000287CD098F80000062873D21C
:10359000DFE800F072030B46464A40F20440008820
:1035A0000390D8F80410814266D098F809104FF0C3
:1035B0000109404601295FD1D0F80A1019B97749AD
:1035C0008969C0F80A100026804617E00720FDF739
:1035D00049FDD7F80E00B846871B402F00D9402779
:1035E000A9193A466E481931FDF7C6FDD8F80A0008
:1035F0003A4630446A4900F015FB3E44D8F80E00C4
:103600004746B042E2D83978012935D14FF0E0225F
:103610000906C2F88011D7F80A0000F0DDF82BE0A7
:103620004FF001092BE086E098F809104FF00109EE
:10363000032924D151495B4A00260B68136016E028
:103640000720FDF70FFDD7F80E00871B402F00D98C
:103650004027A9193A4652481931FDF78DFD4748D0
:103660003A46006881194E48FEF7A0FF3E44D8F85C
:103670000E004746B042E3D898F8180008B1464615
:1036800000E01CE098F80800C00613D54549012267
:1036900003A8C1F800B005F11801CDF80CA0FEF7A1
:1036A00099FF307820B1C8214FF47A70FCF7BDFD46
:1036B000307E20B1307A800701D5FFF738FDD8F889
:1036C0000E001B3505443448FDF7C0FC28B302202A
:1036D0003549A0715D4681F800A00B20FDF7C2FCC2
:1036E000B9F1000F19D04FF00009FDF799F906461E
:1036F00042F21077FDF794F9801BB842FAD34FF4E9
:103700002F714FF47A70FCF790FDFDF76BFA20B93A
:10371000FDF772FA08B9FFF70AFDE078401CC0B265
:10372000E0700C2802D30120A07015E7A0780028D3
:103730003FF414AF10E701202070FFF717FA0120C3
:10374000FFF72CF8184800780028F1D0002106A8CF
:10375000FFF73AFE0028EBD084F806A05D4684F817
:1037600003A0E6E646000000257325640000000083
:103770000CED00E00000FA05A4000010B0000010FD
:10378000940000108C0000109000001055010010F3
:1037900060000010B40000103C010010C4400000A4
:1037A000CD1B0010A800001068000010084A342348
:1037B0001360C2E9010107484FF47A710068B0FB59
:1037C000F1F0D06002F11401104600F05BB8000087
:1037D000101C00100001001072B60349034A01409A
:1037E0001160FCF789BC000080FFFF1F08ED00E0BE
:1037F00010B572B606240E4951F82420824212D91F
:103800000B49783951F82410814207D121460846E6
:1038100000F0E8F821460846FFF7C8FF21460846B1
:1038200000F0E0F802E0641C1D2CE5D962B610BD82
:103830003C41000010B5002821D0114B0022001F90
:10384000196803E0814203D80A4649680029F9D182
:1038500052B11368841A9C4204D100681844106065
:10386000104602E0506000E0186039B102680B1A9F
:10387000934203D10B681A4402604968416010BD4D
:1038800034010010004A1047F11FFF1F214C002592
:10389000FF202560A580A5716071FDF71BF9FDF77C
:1038A000BFF81D4F064600BFFDF7BAF8801BB842AF
:1038B000FAD31A48406B400003D5FFF76BFD00B107
:1038C0006571FEF769F9FCF79FFD70B100F07CF9B6
:1038D00058B10220FDF7C6FB94F90500401C0CD13D
:1038E0000F488069FFF778FF07E00120FDF7BAFB7A
:1038F00094F90500401C00D16571FDF791F8094D60
:10390000044600BFFDF78CF8001BA842FAD3FFF76E
:10391000BDFD0000B4000010A08601000080092059
:10392000C440000080841E00F0B50B30154D20F01F
:1039300007010024144A0FE003688B420BD38B422B
:1039400005D95E1A43184768C3E9006700E0436879
:10395000136002C004E0021D10680028ECD120466C
:10396000002802D1286808B10020F0BD064A0748A7
:103970001060074A121A22F00702C0E90024012051
:103980002860D7E738010010340100107C1D0010BA
:10399000788D0010FFB50246002002EB420501467B
:1039A0004FF440566C4603AA6B1844F82130B342DA
:1039B00002DD002004B0F0BD094F07EB6307DB0711
:1039C0003F78575401D03B095354535C8F0003F0A8
:1039D0000F035354BB40491C18440329E4DBE9E7B7
:1039E00055010010084A32231360C2E9010107485B
:1039F0004FF47A710068B0FBF1F0D06002F114016D
:103A00001046FFF73FBF0000101C0010000100101F
:103A10002DE9F0471D4A00234FF40077156A4FF453
:103A2000FF79C5F30724DFF868A04FF4E05CDFF806
:103A30006480194E25E0B84216D213280CD0142801
:103A40000CD048450CD0A0F58072FF3A0AD03E2831
:103A500013D81AF8002011E0EAB20FE022460DE078
:103A600055220BE0AA2209E0604506D208EB0002CD
:103A7000A2F5805292F8002E00E00022F254401C81
:103A80005B1C8B42D7D3BDE8F087000070000010AC
:103A90008440000055010010CD1B001070B50E468B
:103AA0000546FDF79FF818B9FDF7A6F8002822D0C3
:103AB000B5F5007F1FD32C4CB5F5E05F1CD2FCF7A9
:103AC000AFFFA169401A2949884205D3FCF7A8FF36
:103AD000A06100206060606125490020A1F5D052FE
:103AE00007E02B1813440C5CA3F58053401C83F8AB
:103AF000004EB042F5D370BD606930B9FCF790FF5D
:103B0000A061FCF78DFFA56060611A48407900282C
:103B1000F1D1FCF785FF6169401A174988421DD22F
:103B2000164901200870FCF77BFFA061FCF778FFC5
:103B30006061A0686168281A884203D9616A884276
:103B400000D260600620FDF78DFA61683246BDE85C
:103B50007040074801F50051FEF728BDBDE87040F0
:103B60000C20FDF77FBA000070000010A086010055
:103B7000551B0010B400001020A1070068000010C1
:103B8000FFB50DA60446E1CE8DE8E100022902DA78
:103B9000002004B0F0BD6018002100F8011D694646
:103BA000B3FBF2F502FB1535B3FBF2F34D5D00F804
:103BB000015DA042F4D8ECE730313233343536378A
:103BC000383941424344454646F2044000210088CA
:103BD000A0F51942993A0AD04FF4C0404FF40022A0
:103BE00008C890421944FBD309B100207047012056
:103BF0007047000010B572B63324084B10C307C3DA
:103C000007484FF47A710068B0FBF1F01860191D95
:103C10000248FFF737FE62B610BD0000101C00100E
:103C2000000100102DE9F041144C236803B9206015
:103C30000020134D636803E00F5C1E18401CAF5555
:103C40009042F9D398184FF480766060B04212D158
:103C50002068FFF7CDFD0A4D143D286800B1FEE74E
:103C6000324607492068FFF7C5FF286800B1FEE724
:103C70000020606020600020BDE8F081BC000010E2
:103C8000381C001000050F0A1B1E141133363C3976
:103C9000282D272263666C69787D777250555F5AAC
:103CA0004B4E4441C3C6CCC9D8DDD7D2F0F5FFFA9C
:103CB000EBEEE4E1A0A5AFAABBBEB4B193969C998C
:103CC000888D878283868C89989D9792B0B5BFBA7C
:103CD000ABAEA4A1E0E5EFEAFBFEF4F1D3D6DCD96C
:103CE000C8CDC7C240454F4A5B5E545173767C795C
:103CF000686D676223262C29383D373210151F1A4C
:103D00000B0E040103060C09181D171230353F3A3B
:103D10002B2E242160656F6A7B7E747153565C592B
:103D2000484D4742C0C5CFCADBDED4D1F3F6FCF91B
:103D3000E8EDE7E2A3A6ACA9B8BDB7B290959F9A0B
:103D40008B8E848180858F8A9B9E9491B3B6BCB9FB
:103D5000A8ADA7A2E3E6ECE9F8FDF7F2D0D5DFDAEB
:103D6000CBCEC4C143464C49585D575270757F7ADB
:103D70006B6E646120252F2A3B3E343113161C19CB
:103D8000080D070200002110422063308440A55036
:103D9000C660E770088129914AA16BB18CC1ADD191
:103DA000CEE1EFF13112100273325222B552944239
:103DB000F772D662399318837BB35AA3BDD39CC3E1
:103DC000FFF3DEE36224433420040114E664C77485
:103DD000A44485546AA54BB528850995EEE5CFF531
:103DE000ACC58DD55336722611163006D776F666D9
:103DF0009556B4465BB77AA719973887DFF7FEE781
:103E00009DD7BCC7C448E5588668A77840086118A4
:103E100002282338CCC9EDD98EE9AFF948896999D0
:103E20000AA92BB9F55AD44AB77A966A711A500A78
:103E3000333A122AFDDBDCCBBFFB9EEB799B588B20
:103E40003BBB1AABA66C877CE44CC55C222C033CC4
:103E5000600C411CAEED8FFDECCDCDDD2AAD0BBD70
:103E6000688D499D977EB66ED55EF44E133E322E18
:103E7000511E700E9FFFBEEFDDDFFCCF1BBF3AAFC0
:103E8000599F788F8891A981CAB1EBA10CD12DC11E
:103E90004EF16FE18010A100C230E32004502540B4
:103EA00046706760B9839893FBA3DAB33DC31CD314
:103EB0007FE35EF3B1029012F322D2323542145204
:103EC00077625672EAB5CBA5A89589856EF54FE560
:103ED0002CD50DC5E234C324A01481046674476454
:103EE00024540544DBA7FAB79987B8975FE77EF7B4
:103EF0001DC73CD7D326F2369106B01657667676A4
:103F0000154634564CD96DC90EF92FE9C899E9897F
:103F10008AB9ABA94458654806782768C018E108F3
:103F20008238A3287DCB5CDB3FEB1EFBF98BD89B53
:103F3000BBAB9ABB754A545A376A167AF10AD01A43
:103F4000B32A923A2EFD0FED6CDD4DCDAABD8BAD9F
:103F5000E89DC98D267C076C645C454CA23C832C93
:103F6000E01CC10C1FEF3EFF5DCF7CDF9BAFBABFF3
:103F7000D98FF89F176E367E554E745E932EB23EE3
:103F8000D10EF01E005EBCE2613FDD83C29C7E204C
:103F9000A3FD1F419DC3217FFCA2401E5F01E3BD25
:103FA0003E6082DC237D9FC1421CFEA0E1BF5D0319
:103FB00080DE3C62BEE0025CDF81633D7C22C09E0D
:103FC0001D43A1FF4618FAA427799BC584DA3866F9
:103FD000E5BB5907DB856739BAE406581947A5FBE5
:103FE0007826C49A653BD987045AB8E6A7F91B45D9
:103FF000C6987A24F8A6441A99C7257B3A6486D8CD
:104000005B05E7B98CD2306EEDB3510F4E10F2ACB8
:104010002F7193CD114FADF3702ECC92D38D6F31A4
:10402000B2EC0E50AFF1134DCE90722C6D33D18F98
:104030000C52B0EE326C8ED0530DEFB1F0AE4C128C
:1040400091CF2D73CA947628ABF517490856B4EA78
:104050006937D58B5709EBB536688AD495CB297764
:10406000F4AA4816E9B7550B88D6346A2B7597C958
:104070004A14F6A8742AC896154BA9F7B6E80A544C
:10408000D7896B35EB3C904D53444F53352E300060
:10409000020201000110000004F80C000100010000
:1040A0000000000000000000000029EFBEADDE416E
:1040B000544F4C20465072696E7446415431322040
:1040C0002020000000000000001000000020000080
:1040D00000300000004000000050000000600000C0
:1040E00000700000008000000090000000A00000B0
:1040F00000B0000000C0000000D0000000E00000A0
:1041000000F000000000010000800100000002003B
:104110000080020000000300008003000000040093
:10412000008004000000050000800500000006007B
:10413000008006000000070000800700FF0F00005D
:10414000FF1F0000FF2F0000FF3F0000FF4F000097
:10415000FF5F0000FF6F0000FF7F0000FF8F000087
:10416000FF9F0000FFAF0000FFBF0000FFCF000077
:10417000FFDF0000FFEF0000FFFF0000FF7F0100F6
:10418000FFFF0100FF7F0200FFFF0200FF7F03002F
:10419000FFFF0300FF7F0400FFFF0400FF7F050017
:1041A000FFFF0500FF7F0600FFFF0600FF7F0700FF
:1041B000FFFF0700120110010000004051C203136D
:1041C0000001042048010902200001010080320999
:1041D0000400000208065062070582024000000742
:1041E00005020240000000040309041C03410054BE
:1041F000004F004C00200020002000200020002064
:1042000000200020002000280346005000720069B2
:10421000006E007400200046006C006100730068AE
:104220000020002000200020002000200020001A94
:10423000034600690072006D00770061007200653E
:104240000030003000300030000E034D0065006D7E
:10425000006F007200790000592800000000000083
:104260008D29000000000000000000000000000098
:10427000000000000000000000000000000000003E
:10428000000000000000000000000000000000002E
:104290000000000000000000001BB700BC4200004E
:1042A000000000103C010000D4010000E0420000CA
:1042B0003C0100103C9C0000B4310000A00D4154B2
:1042C0004F4C20465072696E74280549D4284B3DE6
:1042D00002B0104BF902040B14FF0304810000002C
:1042E000C1B78494236130EEA4B7DA9D79088A5D62
:1042F000D783CBB11482FCAB642CF1A69FEE7DB7C3
:10430000053D73B2D35367A12A10BE44855B50B2FA
:10431000ECA00D9C6B65448EA5CFC1E049DFC2C601
:1043200017F0E492CA15D7EABFB576F22D84D5F618
:10433000100288997F8B339C415594789185B6A65D
:10434000DDCE7C4B48E0F1F9F34DCC114D83B73F06
:104350007C8A9160BDCF33E6DB406F2AA3097AB730
:1043600017BD658CD294E05A6DE7973EA026B65DE6
:104370002A818E270D1DF84CF5FA46B5E603F7ABFA
:1043800047BE1D39333FD63A12F0E8DE42E3DBE99F
:10439000243E867C22BB81F9C6F53C6C69AB205D6E
:1043A000B26C1F2F43F238D2D86549F65301C923A6
:1043B0008D4F057A5FC3AC34ED660F9C39262B42D6
:1043C0004368ECD6EF0014B034E4282340FB715C62
:1043D000BFC20407B2EB9469E1C94D02FCC40DEC05
:1043E0005C98F67CE4D8D438FA7A35855712EA21FD
:1043F000D7DE71686578D6AAED47A2C1F769B189A1
:104400001505841801386E11D4DCAF386F3267F8A7
:104410003BDC741EC2A77EED1376EEE38C04B589F7
:104420009BABCAA085612391D9E89328C0B1AF6F37
:10443000C103F555F51367B1451EFDAAB153A7B7E2
:104440003F8A0D551DE5C77F6DEAE24F1C3565A714
:104450004B79593E089D7CB970F886A009DF52F06F
:1044600045F1A16DDA31FB606E1C75E646D0257A08
:1044700024E01D7D1D72415290968C6D14964A5E0B
:10448000E11B03578CC3CEC92D929B269E001A2890
:1044900066C9A32BC5E09CB67A987F9DE364ADA363
:1044A00000066BEBC0C692A588748C8BCE8153AF8F
:1044B00067FFB2088214535CA1C55582D382DAB477
:1044C0005D24EC644E3821EB02B1E0E98668DE5EE3
:1044D000C500BF0A0ED5A7A19609A5B7CD4A164AB1
:1044E000C607A45DE67AAE6BB4A5AE4C74238049D2
:1044F000223889B519197009C048F63C6787B5108C
:104500002C5BFA1107900A68EFCF4C032D56A20BD3
:104510000BBFC2425723F79596F8BC3C684C39391B
:104520004CF1ED29848DF1C7CF843CF7F5AD95BAF8
:104530009A10D4300D1694A4F87EA8C28E8D18332C
:10454000E08A9DD582189AF5FAD42E0B2821A59ED3
:10455000B69763E023BBDEA48A81AA13CAB6B6422B
:10456000BBC980638587CA1D5A3140926B48244F6E
:1045700031EC275B2ADDB72456E4836DE66C874E69
:10458000AA9945A818F4CC72F1AE170C4BD7B60611
:1045900017444E6CC5560D21F282800E263267E715
:1045A000E9577B5D1032A7F63209FE030005496C1E
:1045B00001EE0CB706D876F757A01F2D7DC3212E2C
:1045C0004B5DC557D01BC1B0D520DAC7DFFB42A574
:1045D000CA0E008F9496799EA3CBC20CE9C893446F
:1045E0002B98A9449F2913F566410C7CA7462D837F
:1045F0002E671DE9C2B9802C50021B7B8573C55FF5
:1046000057483A90E8A12354587BA14896A62856CB
:10461000CB7D07C4F5685EF0CBDF504B62FD01A196
:10462000DB78628DA380CA7A8B76090665E89B21C8
:104630002A8EFE4415C6D1BE90D5EDC94494FA1613
:10464000E61A25D3B7E60B9556C291E178FCE21540
:1046500089ACD3606E1F77780EB0829F0306890DF8
:10466000B3C0D8E896E3E9844C771FA4019094EE98
:104670003DDF1839D163E11F92E8BA9BE174C2D3E0
:10468000A21285DB3F96B378BE8D956899D1845090
:104690002A32797EE3CC5A9EACE347156786E06404
:1046A0008D5AC4167F261C3DEBB7165B89E377CD88
:1046B000C741A6C051C309A7582BE1F57E8A83489C
:1046C000C005D15668031BA6EEAE28E94C2737CFAC
:1046D000E43ECEC52C633330D72B83D8FE8939FA1C
:1046E000E56AE43422D5076CE4B6EE6C5747D55939
:1046F00086A4BE007E027FDE61C4C0500C6E09F34A
:1047000079DE058A3C9F1416DEF83CD4DE469D56C1
:104710004741FE834C0A9276D12D2240982A83B7D6
:10472000714E3B2A271E6650832DE321AC2350ADEA
:1047300017BC6B65287452E6388909285F16CC2BA4
:10474000E67C20DFE379C437844F908034EC72C973
:1047500075A7FCFF8C99E68CA2FC41F7016AB02595
:10476000A312C1D7EEFA450C61A85EDAE00D75DA46
:104770005560FD31CD52E372C73A0CC311EFBE6DE7
:10478000101FD2329C9071C35EEED03CF99B07E0C3
:10479000C9622101545B1C038379DFAD24AB2E9BDE
:1047A000B530F198DB4C0C66233473331D6FA0D207
:1047B00051B075518F038DDD2AE82F6B9E8767827C
:1047C000770544F50F3C6F8BB7D745420F095D83E2
:1047D0005D0B767207A13AE3D48F4C90DDC1CBC854
:1047E0002E931F80D2D3A51778CD81AEA285FDF17F
:1047F00094403AC9D7495C37B959AF88DDD8438E60
:10480000EFBDD46ECA311C15E6E6D06350D095AE2C
:104810002DB3091CEAFB9B8750200067F1771837FE
:10482000F7D719061AB872BC4CC39B4903C8EC11E0
:104830000A17C5DB9E928D9AF23E0D5ED523AAE043
:104840003617F1B9FD0AD7F649F729FEF6F12BCD57
:10485000D8060BF69040734EDCA453413CED7562D4
:1048600004B219341FB6F0CEA5AF334BF2622CB1AF
:104870002572D66AB419BF19CA7AB211D79F888334
:104880002824E519F8EF70604DF08CEA2D6411CA08
:10489000CFFDFE18C269C9718F891DFA93155E5349
:1048A0005C995311C1234C876B3400772A45462D00
:1048B00026281364B3C4C72FD6607DCE2CDC361CEB
:1048C000E616D8B61FBD971361284B44243298AE24
:1048D000C74409F889CC325F012C25D91A38E2681F
:1048E000EA31E85CA57FE3B32B69E9F9BAAD593F3A
:1048F000FFD75D6FFED36E65636F8C0A05A2833EA2
:1049000056EB7CFF767F2B4A5A8814CFFB6DE671FD
:10491000CE600F9A5B3C2BBFED923DBAA7A32D2D25
:104920000AECD392754B1F04A892469727841EA1C8
:10493000F812C233AE711723E93F9C90D082BF06B4
:104940002B78696B6A98D654C51BCA20EBB6DFD9A1
:10495000AC79493B1E01E6671231F140D421D00108
:10496000C4F4EDE5A0931D793C1B7C3149CFD0A860
:10497000D32F6EA1420ADBDA6C3F8F21D604F40BF1
:10498000EF2D72952AC78E5346AA8E7B13B2227DD5
:1049900092504E40689754812FD0F16BA488972E87
:1049A00052A445AFBDEF69E44E96FC3B254F6D1A0E
:1049B00027C227632F97492B89A8299FA44CBA5F48
:1049C00042D5021CC50B14CDAD459E93393C6F708A
:1049D0003B5F27DB103F816A8C8DAECBB1E49D2419
:1049E000669C4649E898527878DE7D1750C47088F6
:1049F0009F2E53795B31BED8858994E6140F211D13
:104A00005109A19F0C68E6DAF7D1653F6E7AF65836
:104A10002F3B1D801BC44BB0D98E7E1A29F74D53F6
:104A2000E87CF900068B72ECDE24203B2262262A09
:104A300028C34F86C7C01B4FE9AD1C14D16FABA56F
:104A4000D151801114C9E584354DD9515C9E6A92CB
:104A5000BFBBDBEE11187A856FBEE4618177055329
:104A6000761A135BC5CD17F8C147552E40417B21FF
:104A7000E9904736F66FDB0BA0E38A19548BE6808A
:104A8000636DE7606A3A1AC1F84496F6537947169F
:104A90004AFCE1FA4EEC2756222469C547BD096D50
:104AA000FA5850B339B6C1F252AF630A53A19CCD44
:104AB000ED81BBEFCA34EF2B1B2D31C5E195D3023D
:104AC000A7B64E633AB1BB40624F204C8B59681574
:104AD000BA3AAE17F8F7FCC36ADE98B61E8284783D
:104AE0003B31299C022E84E40BB35F5125E4FFCCBB
:104AF00085A5D5C61BEC5F731F7149ABCCF395C977
:104B0000F20C4FA3407037FB9A76FAF8127E3652B9
:104B100070ABEE659A3FA5B20450C912C3851AD88E
:104B2000823C0F1E496D1EF11F5BABC023FA26426B
:104B300084B7484F9B72829A6CBA20CA1EF0884094
:104B400032BA461A08200C0490EDEC12774866B48D
:104B50005358656279A8A5994B002F6638053D3CEE
:104B6000FC57A0ADE0B972AB3E2E599A17191FA899
:104B70001DC99EA9AAEEA5C8AC6FC628CA128FC6C9
:104B8000EBBC614450B969C821A2550D41DF3B9B84
:104B9000FAFC85DB8918FB465E4E0E33B0C7C32294
:104BA0000AEF853A148F3E37FBA3B9C20F872B1249
:104BB0000FEAA8954A8781B4DD1E4A71EE3B91B990
:104BC000B7E1F8DEABD5FEB9C34E7AB1DE70017C39
:104BD00028E9B2CE27386BB50BDB20FF646E22B418
:104BE0005C8CA49CBC396AB719012AFDF0239DADE9
:104BF000A83149AB81B9F9BFA2D8AB2AD229E99F24
:104C0000C7818D1C12E74C8C6871918128B7A2F383
:104C10007BF680801720B021AA51F1AB5C56BDE134
:104C2000DCE31731AF0D28AE9E4BFFE1FB6B7586C1
:104C3000BB31EC9001DFB1BDBA3C620794B6C1D57F
:104C4000FF77DB16424F5E07850EF0CE7F6D0E4676
:104C500051842B5B014F8E43DCE595164D221F07D7
:104C6000441F456DB46C14CB60D0BB5448068D9581
:104C7000EEAC8C989E4CF83EE99CBF96D21F10601B
:104C80002CC60EC658B2C2A0112905EE4C6EB4EA6D
:104C9000873AEA083F2DED2F87759AA7C1E19A3927
:104CA0007452FE272F18F3F8B89A8E3C19A33E5180
:104CB000BA0AE649E56162EA14BCB04A7BC3CE0099
:104CC0006D866D25DE3BCDBC4DF03288A5FCD6CD82
:104CD0005D8A9E34C5012DFC861BFD74EB7B46204E
:104CE000E40C16048D561C9F3A7AD9C8A2102C5594
:104CF000F91C455A392F0636BDF6919CA6638105ED
:104D00000073AAB91FB4A8F06B7E209E4E19B6118D
:104D100065705845E5C5E7232BDCFC6F23B5B62C41
:104D200060F031EF39DE5FA33D1E3EEA06D107D9C0
:104D3000175A8A91FE89874F4F186AC0C214C092D1
:104D400055A188670E170F96D304470603EC23E49A
:104D5000C00232EE21703189B527B3206666C6FFE6
:104D6000865202A6DED5DD957DF3FB2AD7E3C08807
:104D700078124E0122082C1A2F37CDAA0A199189D0
:104D8000381C96B9D8A7D3B6B133BA07522AEC86E5
:104D9000E6BCBF2802D1F4CA9F0088935FBBE3E75B
:104DA00068DF2029B14D79C013B530B1B0552FCC93
:104DB0008B43331EF9A455CDD99C90F3E13FE5EA2E
:104DC000AE89CB6EEE09F28018A0BF7C99F29D4AA5
:104DD000E994B93CC70A177A1E4EFD342D368AA8CD
:104DE000B81369590DC306B26C381066072594C80C
:104DF0004242236BC24846915981D37979997D52B9
:104E0000530063EA08443E5ADCC76BEB046FD605D7
:104E10001B9C42403874BC3C11CB67F5E0617EAE10
:104E20004473E941EE6C7D49953BF44DA1D80F10D8
:104E300099E7406F242D331A410FBEC2E174A3EFEE
:104E40008131CC46438D802D8F210703632C9EC674
:104E5000C81961C5FF740152F01AA30E796694CF88
:104E6000A682DEA0690FFB8133AF8054DC2073BDC6
:104E700028C6616F903F7D7D93F9FB86FC6298BEEA
:104E8000E0B732C9E441673D4CF76D7E1576277F68
:104E9000CD84FFA2CD1C5E14DD93BBF6990E35F2D6
:104EA000B19D48F1A0BFBE6927B36D833F00DCFF11
:104EB0006CF02E42859AD5076DB3EE651F305B907E
:104EC0007A5A8E6290AA59FF3D23121EFF5FDDA31E
:104ED00048C2C712D0BB17950EA48EE3C490A6AFEC
:104EE0000224947B0F4B24D0B6A8947DC8E7D2C689
:104EF000CB6C92BE7C87AF0685CFDA9344E70BE498
:104F00009A68CBA29B3D7D112C4CDBD35B89D1D71A
:104F100023418F2C46D28E12A5EAF011AF15C0B6F0
:104F20009FEE77125A6F0890B6D567A17ED9F90A1D
:104F30008224CF7595FFC50AA541DBA9490A0CC09B
:104F40000910129943CD5BC8970AB5B53357B68F90
:104F50003BC0AE67FE90EF763970754727055B3C26
:104F60001BA8A2891568C135ECF1F27F6F472C555B
:104F70003E6355A676909F2A199B5ECD3E97662686
:104F800089BCD3752E3CFA6C4424250D4E528DE914
:104F90009922D577840306A297790CAD8D96D964B2
:104FA000757D9B38A7A95083A3597D97BD867DF356
:104FB0001D473A5E2A6B5D574AE7A706D8866E649E
:104FC0009D1A800AB352789327FFB324B25113B9C4
:104FD000575BBB442B650E043C097534CBB7D6B187
:104FE0005719ABB756E6D11B6B1BAE2EEC80F133D5
:104FF00001708B257C24652A721836A62D1D916EB2
:10500000C6EF41324FA5EBD8CAF42551AB9B22B570
:10501000C42951ED1857F92F272C00BFE0D556D4DD
:1050200024B235278FE278347E2DC09AEF272647A9
:1050300060EE8FE62C0D12F00106FEEF55086BE6D0
:1050400051737415F3C53776B7348808A27C496765
:105050008312FDAA2ECBDCB470CFEFAD9A3F3F8018
:105060007BE2818EE77B6620539BF131DD50BDB53D
:1050700004A4BFE5E90CBF2D1B62C5EACDB0FFC299
:1050800067647EC186025BE8E3B2DF6F2390B59070
:105090006D17033B4BF2BD7CAB45A9E8A8D55892F0
:1050A000AAB79A4BAF51241B38B3B18BE05FB97BE1
:1050B00047ADDEB1D41233D2BD7371D30A26EE2BC5
:1050C000B290F2C130D14E2035CFF007CE7413101C
:1050D0005151E2EA54BF7D1F7D5FF72B9D10914532
:1050E000F4C73BD501074690850205786505A00108
:1050F000C9A32EAE1B77231F0A9ED982C0BFD0DA68
:105100009A6F60BEA7B639B8E94F27EECA345AD0B5
:10511000ECB6243EBD4B040E9BC7881AD473051011
:105120007A2E51AE6663D86204C747A894F9D77542
:10513000D6F999F46188D815F8B5EFEFC5866D23D7
:10514000F78B71346E0D502D2CC531262C0D6CBB98
:105150002940FE7B8B56DF34CBEC61F7BD22253036
:1051600012E1E09274A4797F200FC608D5D7896632
:10517000C807F8985C5C0D138348499396F06173F7
:105180007849E1369372E8435A842B887987A523BE
:105190001639380D088439F12326D6A24C0A1C1B77
:1051A000FE64E7AEEEA8D0155201804A74C544CB28
:1051B00044CC200F246EC18314C7BE459CD29EF5FB
:1051C00088743424CEA8C5F724C0A481C147BE4743
:1051D000DF0844DBE05C090E3E0E3BC1A1020AFB86
:1051E000E4F8AA0E26EE12B208225219F0CC2C21B5
:1051F0008C860504793130F30A059A4015DF26497B
:10520000CF4946782B0BC791340913032EE4FDF2E6
:10521000E5A21F098A2C8D0E5EDB73BB7BAF13C723
:10522000BC96BE35594DF2F6B79677EDE4D93931D3
:10523000D4501D66E676C0BD6519B491313D44FD7C
:105240000D28D3CCFF88301013EA8B6BDB563B87DD
:105250000DEBBC37989E46F542E54A022C7131ECC5
:10526000E41A07342A9E8CF6DDCBC67CA4E84F787E
:105270004CAD2A17CD93E7BC888A75795AFC83C256
:10528000EDFD09FDB108989CFB653D370383F0A453
:105290005D443FE4470EDE781747A8B7E6BE0FCC63
:1052A00057ED5722A36B452E8982E6614820A874EA
:1052B0008DB5067ED7E6CFB67382EEBEFDB8F38419
:1052C000C89797A7915B0C66638988DD3B474FAE13
:1052D0002D0D9626D947648BED292741F107EFBDA7
:1052E000DAD496F542D53811BB6E534FC2DE5A342C
:1052F000A663D96E3B543D46A39C9291AFB825E777
:105300007CECDE845886DDA3DBB3663C418441A996
:105310006CCE68EBC003570B0D13ABBED1349DECC4
:10532000D5DB4A96AA429E8ACEE13441A76A317102
:1053300030EFEB4C48BB04A6CE68AC228E671DA2B2
:105340000AD82BB883F0DEAE8985FC5935292F1B8E
:1053500034C49D9239B5E3F8BEA8BE63245C3CF129
:105360001D411E2ECF47B943512C36C1900C6BE224
:10537000A033DC45206106A2B0841040DA68625197
:105380005E3281C3C79C4289347A70CF8D48CE5F2C
:10539000B10E07167C7C02BD6A43347B8D8E25F4EA
:1053A000AA159E39E6868D7DC51DDC77DB1B33563D
:1053B000D2D670ACA87D60AC06D9EFEE50E8C3BB86
:1053C000F9371C9E623444A3ED38F372ED230F8E3F
:1053D000ABE48E2C589EF3A79BEC52B73BD4BBF0AA
:1053E000A3DB248C75BE2164EB6919A751ECEA5D3F
:1053F0001E7516C5DB7B068021482A8E181B760495
:105400006C407387A4FFE2AA9BFA3BF28FCF4A2A33
:10541000FD44F6B445177B7B911E7F53AA61646AF5
:105420000C9E428BD85219FEE8FB65CCD180FB0C58
:10543000362980A1E374452F9662B8FFCF95EF75AA
:1054400049D6F310487F64057FD294CBD959F3D75E
:10545000EF9596687FEB9F8F0077B0DE9B5CE3074C
:10546000CD3BE2A6746395A96D14D0B86BB5021C50
:10547000BD9BF800AA75AF4E7FF2507FB36644A67D
:1054800003B385490A25CF41575943FF11FA0A91C1
:105490005190CBD30E3CB717F94338135EAF1E1EA5
:1054A0009AE34EC8DFC42C257B318AB8C1F38D0B3B
:1054B000EC7D0193CB1279F4067B04626599E0F1EF
:1054C000F4F62514938374C9A5A18CC619D8A482B7
:1054D00064A86116824B3AAA845821A1D5ACD39610
:1054E000FAB1B094F9F37A437A633C4AD03127B0E9
:1054F0003AD94BD6DA0A76F017DB73914F19F103DC
:10550000963BFCA6BA65EB1CCE36611C804F697ACF
:105510005ABEFB07C092FFEB1858CA195657E890BD
:10552000B37EE4826A1205428336E9FB21A58F1817
:1055300077DB8BAAB2D4E81253FFE7C011B3B56A88
:10554000ABF686EA714B41FCAE82D16712DD00AA50
:10555000E29995DAFB4E72C83A93516BD169147394
:10556000D4CDDADC6AF5B988522BF01E6084394E4E
:10557000520B9FEE2B360BEC913B3F27A060B207FE
:10558000C18BBBCDCA17B0A4A0E9E14C6D9A645D94
:105590000E41FBB0DAE04C9C7B94B0F03D05E71C7B
:1055A0006ABC8EDEBA8429F8A3B24AE76A4ABFEA27
:1055B000454908FA349480CA6F15F4C69624D8F881
:1055C0006F8704E3E864415E503CC2A5AB1F94C101
:1055D000CC09655CB57A411272A911885F3DA60CB1
:1055E0000FD39BD72E27C52718D0FDA58D77D6655D
:1055F00044CF211A8770BC2A7F1C5443197627F2A6
:105600009EBB80149A09325C8EC8807CACA171DD8F
:1056100033555345BDAD83215E1785C798C7FFC37A
:105620002C16FE52AF9AC6DC298179405A7375FD5B
:1056300032781A7373908C66B67E78A4B9A5F7ADEC
:10564000F952C0B38CD6EEE9EF434A9E52575A75D1
:10565000A34072977EDB6FDE35CFF84E40B5ECB3DA
:10566000CD1C7BD36A2137317DF8ED4CBC2DE10296
:10567000D3D60768FF8E119574BEABE83B535E40EE
:10568000CF15ECA425212ABC9B5CA4196216859B2E
:105690007319161447EC54920BBCDD56A5DDA3819B
:1056A000741EA77F1FDA86BA09821A8B1D3BC70DAD
:1056B0000E6DFE7A4D963853FA1A24CDF3C6806CDF
:1056C000F6170DBB1668B31ADA95DF0DC41AE16E32
:1056D00019F606D3B7CA5931CF2EF4564D0922FD1B
:1056E00076D4D1EB0A39D6081514B50AE16E3670B6
:1056F0004F3E7AF3850EA501FB1F3238932E2AD830
:105700003939DC62FD7155143AF1C672B913FAF9F0
:105710005A85534E395FB4C71971491F1FBED7CD83
:1057200050CC82E45CE84E7BF1BFA1F03B1FD3D1AB
:10573000650123F5AE279FBDA97E3928B08B4D8624
:10574000FCCA0050DB821D173CD22390AF9474B684
:10575000C2CD605EAF72E198919E1DAA7377DBFFA8
:1057600074F0FA896A70AA1B3B482A0B5631614FC4
:10577000DE8A01CEE544C7B58EE3D0C847A519F748
:105780001ADDC9BB57E1532028880C52768629C8F8
:10579000B8DE897DA5EBA6D0D8263C684D0E6E48B4
:1057A000B439489CF3202E491DB5B408C17A74570A
:1057B000C628EE58386A1FD4AEC3ED16D9B537CF18
:1057C0004F1134F373C7B56C1E28C5708CFF250CC0
:1057D00027F222E570B3727332E2E74F8D9CD09FBF
:1057E0008F2820DCC72BC776F02B757288467B0884
:1057F000ACAE56A108F425CF0D36A8FEE553134DE7
:10580000172BE62B2D4DB4349B2338A2139132561F
:10581000DF207E0E5500A84407129B059B215C15D6
:10582000E1F79ADFFC8DC107BD546EEDC89063EDC2
:105830004FC06923962E0C3CFDDFC866C49C02BC99
:1058400045E0366E9938B4B2C16E3B2EAE6807465D
:105850003D38D899AC19172DBD9745ED2C04A8B249
:105860003B1AC06A25DB010703A177AADA3AD119EE
:105870004955CA779896E91E6198F368C68D5D729E
:105880000556368F45B315711E15C284D734D5978A
:10589000CB9AE145098A515FC9B87BA8AF1FF39342
:1058A000BD8AC4932EFBED4C34BA47BF0D26047A53
:1058B0000DAE650F076DFA1FEE83464AED6DFC676E
:1058C000596F497A47520AE80DFD460A9F324396BE
:1058D0003DB90F7FD067072B7B88BE3CED1572FD6D
:1058E000BA28ADA5BE3231143CE05029726DEC42AD
:1058F0005D14973A8C69447D7C95CA08BA8718DA9A
:10590000B5629CC36E9A3C138AAEF485E0757AFB4F
:105910007842B7366DC56EC4C6861D081C21E68464
:1059200092D2DFE40B4A7C94E7E9449C372922CFEA
:105930004FDBFEB0531F2C7771005D65AA25C5BFF4
:105940000B296A7378324D6633BFC8496E61F00F18
:105950000FAA830ED718E798AAB0CF8631826B17AB
:105960004B79A3F90064929A98F8737B56D8170381
:1059700022CCE87DC3009A0F77D73838FDF709F6B7
:1059800016022E804BF8ED4D5F23F0B67BCDFE3432
:10599000770C93A9BF3AABE7D69C2530E289074D37
:1059A0002699A3AD735D99A9E4344E40861FE7465E
:1059B000BE7D283D5947058BE8D1E8BE24BC616C0B
:1059C00063179182DD9663E23D10BBF4128F0D3AAE
:1059D000F518B02654E9B2D587D4CD9BAE9DF654C8
:1059E0001504FB847E848E9A2FCFF5DA97947E027D
:1059F00007A2AF72FDC6482082D26EC2219563898C
:105A0000C66E4113394F9B3D23C0FF6A93F6EFBD2D
:105A1000C2304B8F1D21C82467130FE2771F5E4FE2
:105A2000E9AE63CDACA90BA17CF1EBFF441621F6E6
:105A30000065366B3B5B679B88AFF1438609BB68AB
:105A4000FE476B9D99F81ED1A08CE6F2EA80B7D78D
:105A500004BE556A9B4D737783E5CA0DD261E7AEEC
:105A60006B2A7F4669FC79F89B1B9ABAC3053F8F66
:105A70002B71A46E56376255FC2B2F69051107D583
:105A800032B686C8E7B01CCD164D91D5F9FC24F886
:105A90002128F9442B282B933E2CE9828C989D1BBE
:105AA000F7D872D925FFCB26F6AA578AAFF0C730B0
:105AB000466E1601AE787F4A4FCD45AFA013AFAF0B
:105AC00041C0F298DB930364A585E4AA3EA7F638AB
:105AD000E3C3728D8CEC6271EAB09C29A5584637FD
:105AE000C308275FF498DFB16DA0CB42A549F0232E
:105AF000D508E0CCE2D89FDE80C08C4F62A4703322
:105B00005BE3B47A98DC016DF492D54B5A12189984
:105B10007DBE6BD8E896AC6E5BCD6899D5E371FA23
:105B2000E65966D6D88108323EF96BC398850A5883
:105B30008412BC6FB4A7421E96E7B8F114D91A8933
:105B40007FBB9CC4E3F45ABDE26F1FDF5DBBF01561
:105B50008E1E0D0D2295393DA9B61F72A142F42E5D
:105B6000EC4B05C92E780827D9135C074A4771C941
:105B7000F28AB78A00F310ED844CD83348218906A5
:105B80004C1702802F88BBC56010027F412A9132DA
:105B90000E8E2FAFE9F482E8FD4F7FFFA34E96F8FB
:105BA0007F89C2CFA783FF967ADFE7EB47FBB2AFCF
:105BB0002B47BDA7AB8EAC91A914D0C27380B23F66
:105BC00090A35FF4C24C900D344BE4EC88CD5E8D15
:105BD000952DC331DAD73088333C3E33D33D7B63D8
:105BE0004B12F0245B1B7B71B8514D584199468490
:105BF000FEB0C6E75FF080AF41E79412ACEBA88639
:105C00000ADF3BA4FACA6F3703E9AF813FF4369548
:105C10008801DDE4428125CB3E53DBA62333F81413
:105C20000DAFC1932D17D3C1530EE8F67B85E0E489
:105C300059E72085D35B4ADC6F15168492811B22BD
:105C400009EA3B8C792A5BE9E1C9F5C01613CCC996
:105C50005EE14E4C46324355C3485C7311CACB7368
:105C60002A5F213FE0B50034B4936D21060189EE2F
:105C7000B8BC27F41910428A526222C495D801F0A8
:105C800074558F980780F2A8ABBA4EE6E63789C202
:105C9000821FE471D9A346122E034B2C3EFD618D69
:105CA0004985D5548131273DEA45935F93B9D95849
:105CB00003A2245405BCBDF8D02BE67A38125A4B07
:105CC000F25E83863CD47A27A462E7D2CAB8CB14AA
:105CD000D3AB067DAE5AB86B2B7E5ACCD1A9C52E5C
:105CE000AC3502888F141CCF3D922C3AC4E78F1C30
:105CF000E7E71EADFC50495F7BB646F571C3DADCC1
:105D0000C44BF85DB8D890A5137921A7B4EF11431F
:105D1000DCEF531A05700BC032FDD956A8AB91BD0C
:105D20004394E3E2F49E04168938044538605E0427
:105D3000A9C2A63066519590C46A813DC8B8B78E95
:105D400049EEAE35480FE12DB5818ED01D52E4D01D
:105D5000AF260535097427D19AEDF4041744CC5FBA
:105D600093C9D9DD98C25C49C2346FD68699A778A9
:105D70002344098494D94B21FCDEBA8B2DA25A56B8
:105D80006657EBAC2DA6B2E65B382334C5C566A1D9
:105D900052175C5E9DC726A08B56EBB9002C445071
:105DA0008993173B51194632BD6F2D70E37DECB3DB
:105DB000AD46F3BE0ECD928132E42807852BA4D8E0
:105DC000F20F58DCF04354FB5D4DFE6D10D15DDCED
:105DD000848041378F373BAC13B17F1884D279A9C7
:105DE000F7428C7914CA5E77BA60A3E3AB65C7B794
:105DF0007236AC4A0885FF3CB0246965B4AF56F3EF
:105E000030FBFD1583FBC251323CCDB56DBC402A41
:105E1000AD38F0C3E66FC54031FED2759BBB4C4434
:105E2000CE072C5970A9851FA3D7F43B572988EAC0
:105E30007DCEC3ADC6D9D2C1DD34013E5181BFCACA
:105E40009CC8FBE84A8D7A2FD126C96CB9439A9039
:105E5000124BEB084D845C325EDC91AB6D8BD38CC6
:105E6000D8A38E056178995746BE35F07D78AF305E
:105E7000CEE884A77E7BF61D70BEB00B65F7B296A8
:105E8000C4C04E10343CF8E7F8781FE36D9DF4462B
:105E9000737598CC376F508D283EF33AE8E8C33DD0
:105EA0004996FFC00BD325B3E689BD07137DB52FF7
:105EB00021E8EE127D129F2237312073457E005B70
:105EC0007FED4273FE4ACA3D9AF10DA384D548C8BE
:105ED0008418A1AE6386305E6EA9BC5252F60BF1F7
:105EE000E1C1ED166A10208773F53B3545E22D833D
:105EF0005BF1F432E5D761B4C655A260F3A59564B1
:105F0000155984C042A98FA27A3232A347DC79C2E4
:105F100063EB7BECFAD9D136526A4A864E9938C582
:105F200045655AD762D0DFAC983F2468202A60913B
:105F3000DD79A548170E24D968A12B088F567DE27C
:105F40003B9EB89A124B4E12BA77E4F17668F1B9DB
:105F50003A1AC617DF7330156FED704CEEA741DFAC
:105F600070D2184555C8AA5C816FA99A4316312290
:105F7000988049F9297367B9AAA95F1CA1C300CC0D
:105F800009DE5CB4530D3A33986AD3B029DF5D6102
:105F9000D559AEF1FEC04E669AF351349F30557A12
:105FA0006417FCEA49CEDDAAF1E7577B83CAD35CCC
:105FB000F796A8B98C168831262C141A6740FAAEC9
:105FC000400CF5760A5AFCC5527D0965B2DF44697A
:105FD00096E4E8A67D53B42DA3B2652C339D8BB017
:105FE0008B4282D1E4B8C2617ECCD0628F0141265F
:105FF000E5939EF283A9E48C8F061BE64358F6DBFB
:00000001FF
